:020000040800F2
:10000000B81D00209D010008FD290008F329000803
:10001000FB2900089D090008252D000800000000AC
:10002000000000000000000000000000AF01000818
:10003000B101000800000000B3010008FF2900081A
:10004000B7010008B7010008B7010008B7010008B0
:10005000B7010008B7010008B7010008B7010008A0
:10006000B7010008B7010008B7010008B701000890
:10007000B7010008B7010008B7010008B701000880
:10008000B7010008B7010008C1080008B70100085F
:10009000B7010008B7010008B7010008B701000860
:1000A000B7010008B7010008B7010008B701000850
:1000B000B7010008B701000800000000B701000800
:1000C000B70100080000000000000000B7010008B0
:1000D00000000000B7010008B7010008B7010008E0
:1000E000B7010008B7010008000000000000000090
:1000F0000000000000000000000000000000000000
:1001000000000000000000000000000000000000EF
:100110000000000000000000752A0008B701000878
:1001200000000000000000000000000000000000CF
:1001300000000000000000000000000000000000BF
:10014000B7010008B701000800000000000000002F
:10015000000000000000000000000000000000009F
:10016000000000000000000000000000000000008F
:10017000000000000000000000000000000000007F
:1001800000000000B7010008DFF80CD000F076FB9B
:100190000048004709390008B81D0020064880477C
:1001A00006480047FEE7FEE7FEE7FEE7FEE7FEE75C
:1001B000FEE7FEE7FEE7FEE70D2A000889010008DA
:1001C000202A04DB203A21FA02F00021704721FAAC
:1001D00002F3D040C2F12002914008431946704713
:1001E00040EA01039B0703D009E008C9121F08C0B9
:1001F000042AFAD203E011F8013B00F8013B521E39
:10020000F9D27047D2B201E000F8012B491EFBD2AF
:1002100070470022F6E710B513460A460446194611
:10022000FFF7F0FF204610BD2DE9FE4F804681EA22
:100230000300C00F0C46009021F0004123F0004560
:10024000B8EB0200A94105D24046214690461C4623
:100250000B46024623F00040104347D0270DC7F35A
:100260000A00C3F30A510290401A019040286BDA49
:10027000C3F3130040F4801B0098924620B1002382
:10028000D2EB030A63EB0B0B01985946C0F1400215
:10029000504600F08DF906460D4650465946019AE3
:1002A00000F095F910EB08006141002487EA115233
:1002B00084EAE7731A4340D0009A62B3019A012A94
:1002C0004FEA075215DC001B61EB02014FF00042C0
:1002D00002EA0752CDE90042001C41F58011324686
:1002E0002B4600F0CCF903B0BDE8F08F4046214624
:1002F000F9E7001B61EB0201001C41F580130018B7
:100300005B412018A2F5001747EB030140EAD570C6
:10031000B6196D4111E06D084FEA360645EAC07521
:100320004FEA0752001B61EB0201001C41F58011EE
:1003300049084FEA30000019514132462B4603B0BC
:10034000BDE8F04F00F08CB9009801224000002376
:10035000D0EB020263EBE073009821464FEAE074B1
:10036000B8EB000061EB0401E9E783F000435BE7D1
:1003700081F0004158E72DE9FE4F81EA030404F0C3
:10038000004421F0004100944FF0000B23F00043A3
:1003900050EA01045ED052EA03045BD0C3F30A546E
:1003A000C1F30A552C44A4F2F3340194A0FB025487
:1003B000C1F3130141F48011C3F3130343F4801319
:1003C00001FB024400FB034E840A970A44EA81546D
:1003D00047EA8357A4FB076802958D0A05FB07854A
:1003E0004FEA932C04FB0C542705029D4FEA065854
:1003F00047EA1637B5EB08056EEB070C870E920E31
:1004000047EA811742EA8312A7FB0201B6EB0B0110
:1004100064EB00042B0D43EA0C335E1844EB1C50D4
:10042000DA465146E7FB0201C5F313044FEA0B33EA
:1004300043EA14534FEA0432019C43EA0603A4F151
:100440000C040294009CCDE900B400F018F903B04C
:10045000BDE8F08F00200146F9E72DE9F04D81EA73
:10046000030404F0004B21F0004514464FF0000A4D
:1004700023F0004150EA050220D054EA01021DD0C9
:10048000C5F30A570246C5F31303C1F31300C1F3C2
:100490000A5640F4801543F48013A7EB0608101B9E
:1004A000D64608F2FD3873EB050002D308F10108C7
:1004B00001E092185B41B8F1000F03DA0020014619
:1004C000BDE8F08D00204FF48011064684460EE012
:1004D000171B73EB050705D3121B63EB05030643DC
:1004E0004CEA010C49084FEA300092185B4150EA8F
:1004F0000107EDD152EA030012D082EA040083EA38
:100500000501084305D0101BAB4106D20122002390
:1005100006E000224FF0004302E06FF001025310AA
:100520001AEB06004CEB085110EB0A0041EB0B01F3
:10053000BDE8F04D00F094B80EB540F233410291A1
:100540000021CDE900110A460B4600F098F803B0EF
:1005500000BD00F0004230F000400AD0C10D01F5AE
:100560006071C0F3160042EA0151C208400711430E
:10057000704700200146704701F0004330B421F07D
:10058000004150EA010206D00A0DA2F56072C1F3E3
:100590001301002A02DC30BC00207047440F44EAFB
:1005A000C104C100E01830BC00EBC25000F021B81B
:1005B000202A04DB203A00FA02F100207047914023
:1005C000C2F1200320FA03F3194390407047202A18
:1005D00006DBCB17203A41FA02F043EAE07306E06B
:1005E00041FA02F3D040C2F120029140084319467B
:1005F00070470029A8BF7047401C490008BF20F081
:100600000100704710B4B0FA80FC00FA0CF050EA18
:10061000010404BF10BC704749B1CCF1200421FA99
:1006200004F411FA0CF118BF012121430843A3EB94
:100630000C01CB1D4FEA00614FEA102042BF0020A1
:1006400010BC704700EBC35010440029A4BF10BC7D
:100650007047401C490008BF20F0010010BC7047E3
:1006600010B5141E73F1000408DA401C41F10001BA
:1006700092185B411A4301D120F0010010BD2DE911
:10068000F04D92469B4611B1B1FA81F202E0B0FA08
:1006900080F220329046FFF78BFF04460F4640EA77
:1006A0000A0041EA0B0153465A46084313D011464B
:1006B00053EA010019D0C8F140025046FFF780FD0F
:1006C00005460E46504659464246FFF771FF08431D
:1006D00005D0012004E020463946BDE8F08D002019
:1006E000054346EAE0762C4337430A986305E40A5B
:1006F000A0EB08000022FD0A44EA47540A3002D564
:1007000000200146E9E7010510196941DDE90845C6
:1007100000196941BDE8F04DA2E72DE9F04D002335
:100720001A461B1A8A4103DB00200146BDE8F08D02
:10073000C1F30A52C1F3130141F480154FF0000BCD
:10074000D10702D100186D41521E0027044640F225
:10075000FF11384601EB620A3E4680460246002001
:100760004FF48011FFF72CFDC2197141BB1846EB05
:100770000100B4EB030C75EB000C04D3E41A65EB39
:10078000000517460E46241908F101006D41804608
:100790003428E3DDF91946EB0600091BA84103D212
:1007A0004FF0FF32134601E0002213461BEB070017
:1007B00046EB0A51BDE8F04DFFF752BF0EB5C10F31
:1007C00080EAE0700844CA07002140F233438DE814
:1007D0000E000A460B46FFF752FF03B000BD70B58E
:1007E000C1F30A5201F000450024C1F3130140F2A5
:1007F000FF3341F480119A4201DA002070BD40F2CB
:1008000033439A42A2F2334203DC5242FFF7D8FC50
:1008100000E090402C43F1D0404270BD30B5041E42
:1008200071F1000404DB4FF00044404264EB01012D
:10083000141E73F1000405DB1C464FF000435242C6
:1008400063EB04038B4208BF824230BD30B5041E07
:1008500071F1000404DB4FF00044404264EB0101FD
:10086000141E73F1000405DB1C464FF00043524296
:1008700063EB0403994208BF904230BD064C074D1C
:1008800006E0E06840F0010394E807009847103460
:10089000AC42F6D3FFF77CFCE8420008184300089E
:1008A00040F2B12CC1F2000C604740F2E31CC1F2EF
:1008B000000C604740F2C56CC1F2000C60470000BC
:1008C000014800F033BA00001801002070B504465A
:1008D0000068816801F0030101292BD1016811F042
:1008E000010F27D0816801F00D01012913D1816822
:1008F00041F00201816021680320086001F04EF898
:1009000005462068806810F0010F13D001F046F80A
:10091000401B022809D9606C40F010006064A06C94
:1009200040F00100A064012070BD2068806810F0D4
:10093000010FEBD1002070BD70B5044600688168DE
:1009400001F00301012903D1016811F0010F23D146
:1009500081686FF39E1181B9816841F00101816066
:1009600001F01CF805462068006810F0010F13D153
:1009700001F014F8401B022809D9606C40F0100007
:100980006064A06C40F00100A064012070BD20688C
:10099000006810F0010FEBD0002070BDFEE7FEE70D
:1009A00070477047704770472DE9F00198B04FF0DD
:1009B000000CCDF808C090F840206446012A01BF21
:1009C000022018B0BDE8F0017047012780F84070A0
:1009D0000268936813F0040F40F04A814B681F25AA
:1009E000052B0CD2166B03EB43035B009D4026EAFC
:1009F00005050E6806FA03F32B4313632CE00A2B5C
:100A00000DD2566B5B1F03EB43035B009D4026EA50
:100A100005050E6806FA03F32B4353631CE00F2B06
:100A20000DD2966B0A3B03EB43035B009D4026EA25
:100A300005050E6806FA03F32B4393630CE0D66BAF
:100A40000F3B03EB43035B009D4026EA05050E6860
:100A500006FA03F32B43D363026893684FF007054C
:100A600013F00C0F64D10B680A2B0ED396690A3B66
:100A700003EB430305FA03F826EA0806D1F80880D9
:100A800008FA03F3334393610CE0566903EB430325
:100A900005FA03F826EA0806D1F8088008FA03F3F5
:100AA0003343536102684B69D668D1F81080C6F3AE
:100AB000C1067600B340974EB8F1010F3FD0B8F1B0
:100AC000020F49D0B8F1030F53D0B8F1040F5DD035
:100AD000136E0E7803F0F843B3EB866F03D1136EF9
:100AE00023F0004313660268536E0E7803F0F84358
:100AF000B3EB866F03D1536E23F000435366026855
:100B0000936E0E7803F0F843B3EB866F03D1936EC8
:100B100023F0004393660268D36E0E7803F0F84327
:100B2000B3EB866F04BFD36E23F0004300D1D366CE
:100B30000268936803F00303012B37D132E0D2F847
:100B4000608008EA060691F8008043EA8863334330
:100B500043F000431366EBE7D2F8648008EA060628
:100B600091F8008043EA8863334343F000435366BF
:100B7000DEE7D2F8688008EA060691F8008043EACA
:100B80008863334343F000439366D1E7D2F86C8027
:100B900008EA060691F8008043EA8863334343F08D
:100BA0000043C4E7136813F0010F67D1CB68012B32
:100BB000D2F8B03006D00D7807FA05F5AB43C2F88D
:100BC000B03022E00E7807FA06F63343C2F8B030B0
:100BD0000A6803680A2A0CD39E69093A02EB4202AA
:100BE000954026EA05058E6806FA02F22A439A61C4
:100BF0000BE05E69521C02EB4202954026EA0505B5
:100C00008E6806FA02F22A435A610968424A10299C
:100C100008D011290BD0122904BF936813F4800F58
:100C200009D02BE0936813F4000F27D103E09368F9
:100C300013F0807F22D10368B3F1A04F0CBF374D72
:100C40004FF0A04503959D6805F00305012D03D1E4
:100C50001D6815F0010F0BD1039DB5B1AD6805F00E
:100C60000305012D11D1039D2D6815F0010F0CD046
:100C7000416C41F0200141644FF0010C80F840408C
:100C800018B06046BDE8F0017047102909D011295D
:100C900033D0122904BF916841F48001EED19160F4
:100CA000ECE7B3F1A04FE9D1916841F40001916004
:100CB0001B491C4A0968B1FBF2F101EB81014900B3
:100CC00002910091DAD0B1F1004F1ED20029D8BFB5
:100CD000002105DD11F0010102D0029A521E02929C
:100CE000009A491C531C9942C8DA029A891C521E68
:100CF000521E02929942F8DBC0E7B3F1A04F04BF45
:100D0000916841F08071B9D1C9E70299491E0291F9
:100D1000FCD1B3E700F0FF83000300500001005056
:100D20000400002040420F007047704770B5044631
:100D3000006801684FF0A04511F0040F1CBF416826
:100D400011F0040F04D0616C11F0100F0DD108E008
:100D5000016811F0080F1CBF416811F0080FF2D1B3
:100D600038E0616C41F400716164D5F8081311F04A
:100D70001F0F17D0D5F8081301F01F01052911D056
:100D8000D5F8081301F01F0109291CBFB0F1A04FCD
:100D9000E96807D0C26812F4406F08BF11F4005F21
:100DA00012D101E0C168F5E7016811F0080F0BD01E
:100DB000816811F0040F3DD0606C40F01000606459
:100DC000A06C40F00100A0642046FFF7ADFF216851
:100DD0000C2008602068016811F0200F1CBF4168DA
:100DE00011F0200F37D0616C41F400516164D5F8E7
:100DF000081311F01F0F37D0D5F8081301F01F01A9
:100E0000052931D0D5F8081301F01F0109291CBFAD
:100E1000B0F1A04FE96827D0C26C12F0C00F25D006
:100E200011F0007F02BFC26812F4406F11F4005F3E
:100E30001CD047E0416821F00C014160606C20F457
:100E400080706064606C10F4805FBDD1606C40F0B5
:100E500001006064B8E7016811F0400F1CBF4168F1
:100E600011F0400FBFD133E0C168D5E7016811F040
:100E7000400F27D0D5F8081311F01F0F14D0D5F864
:100E8000081301F01F0106290ED0D5F8081301F050
:100E90001F0107291CBFB0F1A04FE96804D000BFB3
:100EA00011F4001F02D00DE0C168F9E7816811F06C
:100EB000080F7DD0606C40F010006064A06C40F0C2
:100EC0000100A0642046FFF76BFD216860200860E8
:100ED0002068016811F0800F1CBF406810F0800F7F
:100EE00009D0606C40F480306064204600F09EF9C8
:100EF0002168802008602068016811F4807F1CBF91
:100F0000406810F4807F0AD0606C40F40030606468
:100F10002046FFF747FD21684FF480700860206885
:100F2000016811F4007F1CBF406810F4007F0AD0F4
:100F3000606C40F4802060642046FFF734FD216837
:100F40004FF4007008602168086810F0100F1CBF93
:100F5000486810F0100F19D0A06B012808D0244861
:100F6000826812F01F0F3DD0806810F4404F0AD005
:100F7000606C40F480606064A06C40F00200A0648B
:100F80002046FFF7D2FE2168102008602068016823
:100F900011F4806F1ABF416811F4806F70BD616CED
:100FA00041F480416164A16C41F00801A16400E05A
:100FB00006E04FF4806101602046FFF7F2FC70BD4F
:100FC000416821F060014160606C20F480506064F1
:100FD000606C10F4807F7FF475AF606C40F00100AE
:100FE00060646FE7C86810F0010FC1D1CBE7000063
:100FF0000003005070B596B04FF00006040035466F
:10100000029602BF012016B070BD606C10F0100F88
:10101000606C03D010F0100F69D06DE000284BD148
:10102000A5642565E56484F84050204600F000F989
:101030002068806810F0805F3ED12046FFF746FCB4
:101040000646606C10F0100F08BF002E34D1606CA3
:1010500020F4885040F0020060642068816821F02C
:10106000405181602068816841F080518160694809
:1010700069490068B0FBF1F000EB8000400002908D
:10108000009019D0B0F1004F80F0BE800028D8BF8A
:10109000002005DD10F0010002D00299491E0291E6
:1010A0000099401C491C884206DA029A801C521E94
:1010B000521E02928842F8DB2068816811F0805F3E
:1010C00003D0806810F0005F0BD0606C20F002004D
:1010D00040F010006064A06C40F00100A064606CFF
:1010E0000AE0606C10F0100F08BF002E04D12068D9
:1010F000816811F0040F0AD0606C20F0020040F00B
:10110000100060644FF0010616B0304670BD616C8F
:1011100021F4807141F0020161644049B0F1A04FB7
:1011200014BF4FF0A0423E4A0092826802F00302D0
:10113000012A03D1006810F0010F11D1009848B1C5
:10114000806800F00300012804D10098006810F0C6
:10115000010F05D18868626820F440301043886030
:10116000D4E902100843A16B012914BF4FF4805247
:101170000022E16942EA41321043626A012A0AD13F
:10118000A9B1616C21F0020141F020016164A16C00
:1011900041F00101A164E16A012902D0226B1143EF
:1011A000084321688A6812F00C0F14D107E0218DE2
:1011B0001C4A02EB4141084340F48030EBE7CA6827
:1011C00022F0020222F48042CA60A169626B8903A4
:1011D00041EA420108432168CA68134B1A40104390
:1011E000C860206901282068016B21F00F0102D13D
:1011F000226A521E11430163A564606C20F0020054
:1012000040F0010060647FE70298401E0290FCD12C
:1012100052E700000400002040420F00000300508D
:10122000000100500000FEFF07C0F0FF7047000003
:1012300000B5006887B0B0F1A04F1CBF07B000BD7B
:101240000D48416941F0805141614069694600F0B3
:1012500080500590032000900190002002900748E4
:1012600000F08CFA00221146122000F01BFC122024
:1012700000F00CFC07B000BD001002400004004864
:101280002DE9F047044640690F464FF00009082851
:1012900008BF082519D03948816811F01F0F0DD0FB
:1012A000806810F4404F0ED0606C40F02000606405
:1012B00084F840904FF00100BDE8F0872068C068D6
:1012C00010F0010FF0D14FF00C054FF0A040D0F816
:1012D000081311F01F0F1ABF2168B1F1A04F206849
:1012E000C66800F05BFB804620680068284216D183
:1012F000B7F1FF3F0FD02FB100F050FBA0EB08007B
:10130000B84208D9606C40F00400606484F84090F2
:101310000320BDE8F087206800682842E8D0606CB0
:1013200040F4007060642068C16811F4406F08BF29
:1013300016F4005F0FD1016811F0080F0BD081681F
:1013400011F0040F616C0DD041F020016164A16CBB
:1013500041F00101A16416F4804F08BF0560002030
:10136000BDE8F08721F480716164616C11F4805FE5
:10137000F1D1616C41F001016164ECE700030050C0
:1013800010B504460068806810F0040F18BF0221F1
:1013900001D0084610BD94F84000012804BF022087
:1013A00010BD012084F840002046FFF7C5FA010077
:1013B0004FF0000218BF84F84020EAD1606C20F0A2
:1013C000010020F4606040F4807060644FF0A04041
:1013D000D0F8083313F01F0F1CBF2368B3F1A04FE0
:1013E0003ED0D4F844C04CF4801CC4F844C0A3F1EF
:1013F000A04CBCF5807C09D1C36813F0007F05D0F8
:10140000636C23F4005343F480536364636C13F4FC
:10141000805F08BFA26403D0A36C23F00603A3641B
:1014200084F8402023681C221A60D0F8082312F0A8
:101430001F0F0FD0D0F8082302F01F02052A09D091
:10144000D0F8080300F01F0009281CBF2068B0F185
:10145000A04F9ED12068826842F00402826098E723
:10146000636C23F4801363642368DB6813F0007FEC
:10147000C6D1CBE7002804BF0120704790F82110A7
:101480000023002908BF80F8203030B4022180F802
:10149000211002681168D0E901C44CEA040CD0E9BB
:1014A00003452C434CEA040C44696FF30D114CEADC
:1014B000040C84694CEA040CC4694CEA040C4CEA40
:1014C000010111608363012180F8211030BC0020EC
:1014D000704700002DE9F74F82B004460399884E0B
:1014E000DFF820B2DFF82082DFF820920068924611
:1014F000002977D0B04208BF04271AD0584508BF4A
:10150000402716D0404508BF4FF4806711D04845AA
:1015100008BF4FF480470CD07D49884208BF4FF484
:10152000802706D07B4988420CBF4FF480074FF0DC
:10153000806700F033FA784D00902868384271D106
:1015400029682068B04208BF08221AD0584508BF51
:10155000802216D0404508BF4FF4006211D04845A4
:1015600008BF4FF400420CD0694A904208BF4FF4C4
:10157000002206D0674A90420CBF4FF400024FF0A1
:10158000006211424FD0B04208BF08201AD058451F
:1015900008BF802016D0404508BF4FF4006011D02E
:1015A000484508BF4FF400400CD05949884208BF55
:1015B0004FF4002006D0574988420CBF4FF400007A
:1015C0004FF000606860A06B40F00100A063042051
:1015D00084F82100002084F8200005B00120BDE837
:1015E000F08FFFE7B04208BF0227A2D0584508BFDE
:1015F00020279ED0404508BF4FF4007799D048453A
:1016000008BF4FF4005794D04149884208BF4FF4B7
:1016100000378ED03F4988420CBF4FF400174FF07F
:10162000007786E71DE0BAF1FF3F16D0BAF1000F50
:1016300005D000F0B3F90099401A50450DD9A06BC0
:1016400040F02000A063032084F82100002084F8EB
:10165000200005B00320BDE8F08F286838423FF431
:101660006FAF03980028206828D0B04208BF04203C
:101670001AD0584508BF402016D0404508BF4FF447
:10168000806011D0484508BF4FF480400CD02049FD
:10169000884208BF4FF4802006D01E4988420CBF04
:1016A0004FF480004FF080606860112084F82100C2
:1016B000002084F8200005B0BDE8F08FB04208BFDC
:1016C00002201AD0584508BF202016D0404508BF38
:1016D0004FF4007011D0484508BF4FF400500CD0B3
:1016E0000B49884208BF4FF4003006D009498842B0
:1016F0000CBF4FF400104FF0007068600120D5E778
:10170000080002401C000240300002404400024039
:10171000580002406C0002400000024090F820C0D7
:10172000BCF1010F04BF0220704710B44FF0010C50
:1017300080F820C04FF0020C80F821C0D0F800C023
:10174000DCF8004024F00104CCF80040D0F800C0E0
:10175000CCF804304368102B036803BF9A6002681A
:10176000D16099601CBF0168CA600068016841F0DF
:101770000101016010BC0020704700000B680022CE
:10178000002B08BF70472DE9F84F784EDFF8E0E1F5
:1017900001274FF0030A4FF00F0800BF0B6807FA4C
:1017A00002F52B407ED0D1F804C0BCF1020F18BF67
:1017B000BCF1120F15D14FEAD20C00EB8C04D4F817
:1017C00020904FEA427C4FEADC6C08FA0CFB29EAD5
:1017D0000B09D1F810B00BFA0CFC4CEA090CC4F858
:1017E00020C0D0F800904FEA420C91F804B00AFAF9
:1017F0000CF40BF0030B29EA04090BFA0CFB4BEA7F
:101800000909C0F80090D1F80490B9F1010F18BF90
:10181000B9F1020F05D0B9F1110F18BFB9F1120FCC
:1018200018D1D0F80890D1F80CB029EA04090BFAC5
:101830000CFB4BEA0909C0F80890D0F8049029EA9B
:10184000050591F80490C9F3001909FA02F949EA6B
:1018500005054560C56825EA04048D6805FA0CFC99
:101860004CEA040CC0F80CC0D1F804C01CF0805F36
:1018700075D0D6F818C04CF0010CC6F818C0D6F8D0
:1018800018C00CF0010CCDF800C022F0030C0CF1D4
:10189000804404F58034D4F808C04FEA82754FEADA
:1018A000157500E05BE008FA05F92CEA090CB0F1C7
:1018B000904F08BF4FF0000918D0A0F19049B9F53A
:1018C000806908BF4FF0010910D0A0F19049B9F527
:1018D000006908BF4FF0020908D0A0F19049B9F59E
:1018E00040690CBF4FF003094FF0050909FA05F5EF
:1018F00045EA0C0CC4F808C0DEF800C04C682CEABD
:10190000030C14F4803F18BF4CEA030CCEF800C05F
:10191000184CD4F800C04D682CEA030C15F4003FB5
:1019200018BF4CEA030CC4F800C0134CD4F800C034
:101930004D682CEA030C15F4801F18BF4CEA030C09
:10194000C4F800C00D4CD4F800C04D682CEA030C5C
:1019500015F4001F18BF4CEA030CC4F800C00B6854
:10196000521CD3407FF41AAFBDE8F88F001002403C
:101970000004014004040140080401400C0401403B
:101980000069084018BF0120704742695140416119
:101990007047002A14BF8161816270470148006866
:1019A000704700000000002002480168491C0160E7
:1019B0007047000000000020074810B5016841F0A2
:1019C00010010160032000F09FF8002000F006F8ED
:1019D00000F018F8002010BD0020024010B50446A9
:1019E00007484FF47A720068B0FBF2F000F0DCFCBC
:1019F00000222146501E00F055F8002010BD0000C6
:101A0000040000201A4808B5816941F00101816194
:101A1000806900F001000090032000F075F80022BA
:101A200011466FF00B0000F03DF8002211466FF0F8
:101A30000A0000F037F8002211466FF0090000F0AC
:101A400031F800221146501F00F02CF800221146F8
:101A5000101F00F027F800221146901E00F022F817
:101A60000022BDE808401146501E00F01BB80000DF
:101A70000010024000F01F01012202FA01F14009AA
:101A8000800000F1E020C0F88011704700F01F01D5
:101A9000012202FA01F14009800000F1E020C0F8C3
:101AA00000117047174B10B41B68C3F30223C3F136
:101AB000070CBCF1040F88BF4FF0040C1C1D072C51
:101AC00034BF0023DB1E012404FA0CFCACF1010C32
:101AD0000CEA0101994004FA03F35B1E1A4011431A
:101AE00000284FEA0111A1BF00F1E02080F80014A6
:101AF00010BC704700F00F0000F1E02080F8141DCA
:101B000010BC70470CED00E0074900F007000A68C0
:101B10004FF6FF031A4042EA002040F0FD7040F00B
:101B200080600860704700000CED00E0BFF34F8F4D
:101B300005480168054A01F4E06111430160BFF303
:101B40004F8F00BFFDE700000CED00E00400FA0538
:101B50000548016841F0020101600448016841F054
:101B60000401016030BF70470070004010ED00E0DC
:101B70002DE9F047DFF8289205460E46D9F8000017
:101B800000F00700B0420CD2D9F8000020F00700A6
:101B90003043C9F80000D9F8000000F00700B04257
:101BA00070D128787F4C10F0020F05D06068A968CA
:101BB00020F0F00008436060287810F0010F71D029
:101BC00068680121012831D0022845D0022393FA08
:101BD000A3F2B2FA82F242F0200252090CBF626A0A
:101BE000226893FAA3F3B3FA83F303F01F03994037
:101BF0000A427DD0616821F0030108436060FFF76D
:101C0000CDFE0746686841F2883801283BD002289B
:101C1000606800F00C0046D0002856D0FFF7BEFEEA
:101C2000C01B40454DD90320BDE8F0874FF4003379
:101C300093FAA3F2B2FA82F242F02002520914BFE0
:101C40002268626A93FAA3F3B3FA83F303F01F03E3
:101C500099400A424CD0CDE74FF0007393FAA3F2BB
:101C6000B2FA82F242F02002520914BF2268626A7C
:101C700093FAA3F3B3FA83F303F01F0399400A42E4
:101C800036D0B7E734E0606800F00C0004281CD0C0
:101C9000FFF784FEC01B4045C5D8606800F00C000B
:101CA0000428F5D111E008280FD000BFFFF776FE19
:101CB000C01B4045B7D8606800F00C000828F5D17B
:101CC00003E0606810F00C0FA8D1D9F8000000F014
:101CD0000700B0420FD9D9F8000020F007003043C8
:101CE000C9F80000D9F8000000F00700B04202D0A7
:101CF0000120BDE8F087287810F0040F05D0606857
:101D0000E96820F4E06008436060287810F0080F6C
:101D100006D06068296920F4605040EAC100606024
:101D20006168214801F00C02042A01D0082A13D06E
:101D30006168F02292FAA2F201F0F001B2FA82F2A6
:101D4000D1401A4A515CC840194908600020FFF789
:101D500045FE0020BDE8F0874FF4701393FAA3F31B
:101D600001F47012B3FA83F3DA40124B9A5CE36A1F
:101D70004FF00F0C9CFAACFC03F00F03BCFA8CFC88
:101D800023FA0CF3DFF830C011F4803F1CF8033065
:101D900019BFB0FBF3F0504308485043C8E70000B8
:101DA000002002400010024000127A00A441000806
:101DB00004000020844100089441000800093D000F
:101DC0000148006870470000040000202DE9F84F2A
:101DD00004460078FF4D10F0010F4FF0010626D0A9
:101DE0006868770400F00C00042808D0686800F0E8
:101DF0000C00082860D1686810F4803F5CD097FA26
:101E0000A7F0B0FA80F040F02000400914BF286825
:101E1000686A97FAA7F1B1FA81F101F01F0106FA99
:101E200001F1084203D06068002800F0AA822078FF
:101E30004FF0000910F0020F4FF0020778D06868E9
:101E40004FF0F80A10F00C0F73D0686800F00C0027
:101E5000082804BF686810F4803F6AD02069002811
:101E600096FAA6F0B0FA80F04FEA800000F18440C4
:101E700000F5840000F0F8800660FFF78FFD8046D3
:101E800097FAA7F0B0FA80F040F02000400914BFA4
:101E90002868686A97FAA7F1B1FA81F101F01F0189
:101EA00006FA01F108426ED1FFF778FDA0EB0800B9
:101EB0000228E5D900F013BA6068B0F5803F04BF8E
:101EC000286840F480300AD010B1B0F5A02F31D08E
:101ED000286820F480302860286820F4802028605A
:101EE000E86AA16820F00F000843E862606848B320
:101EF000FFF754FD4FEA000897FAA7F0B0FA80F018
:101F000040F02000400914BF2868686A97FAA7F1DA
:101F1000B1FA81F101F01F0106FA01F1084286D100
:101F2000FFF73CFDA0EB08006428E5D900F0D7B925
:101F30005CE029E0286840F480202860286840F4AC
:101F40008030CCE7FFF72AFD4FEA000897FAA7F0A8
:101F5000B0FA80F040F02000400914BF2868686A99
:101F600097FAA7F1B1FA81F101F01F0106FA01F128
:101F700008423FF45CAFFFF711FDA0EB08006428B6
:101F8000E4D900F0ACB924E097FAA7F0B0FA80F0F9
:101F900040F02000400914BF2868686A97FAA7F14A
:101FA000B1FA81F101F01F0106FA01F108421CBFEC
:101FB0002069012840F0E58128689AFAAAF261694F
:101FC000B2FA82F220F0F80001FA02F140EA0100D0
:101FD0000BE028689AFAAAF220F0F8016069B2FAD8
:101FE00082F200FA02F041EA00002860207810F046
:101FF000080F7CD0A069002896FAA6F0B0FA80F00D
:102000004FEA800000F1844000F584004ED0C0F813
:102010008064FFF7C3FC804697FAA7F0B0FA80F01F
:1020200040F06000B6EB501F08BF28680AD097FA4E
:10203000A7F0B0FA80F040F06000B7EB501F0CBF83
:10204000286A686A97FAA7F1B1FA81F101F01F01D5
:1020500006FA01F1084258D1FFF7A0FCA0EB0800F6
:102060000228D9D900F03BB9C0F80090FFF796FCE0
:102070004FEA000897FAA7F0B0FA80F040F020008D
:10208000400914BF2968696A97FAA7F0B0FA80F08E
:1020900000F01F0006FA00F00142A7D0FFF77EFC17
:1020A000A0EB08000228E5D900F019B9C0F8809427
:1020B000FFF774FC4FEA000897FAA7F0B0FA80F037
:1020C00040F06000B6EB501F08BF28680AD097FAAE
:1020D000A7F0B0FA80F040F06000B7EB501F0CBFE3
:1020E000286A686A97FAA7F1B1FA81F100E00CE07A
:1020F00001F01F0106FA01F1084206D0FFF74EFC7D
:10210000A0EB08000228D7D9E9E0207810F0040FEE
:102110005FD0E8694FF0000B10F0805F09D1E869EB
:1021200040F08050E861E8694FF0010B00F080500A
:102130000090DFF8A480D8F8000010F4807F18D158
:10214000D8F8000040F48070C8F80000FFF726FCC3
:102150008246D8F8000010F4807F0AD1FFF71EFCF9
:10216000A0EB0A00642849D8D8F8000010F4807F5A
:10217000F4D0E068012804BF286A40F0010009D0CB
:1021800008B105283CD0286A20F001002862286A9E
:1021900020F004002862E06841F2883A78B3FFF743
:1021A000FDFB804697FAA7F0B0FA80F040F04000BF
:1021B000B6EB501F08BF28680AD097FAA7F0B0FA0C
:1021C00080F040F04000B7EB501F0CBF286A686AEF
:1021D00004E04FE0001002400070004097FAA7F1C1
:1021E000B1FA81F101F01F0106FA01F108423AD17A
:1021F000FFF7D4FBA0EB08005045D3D96FE007E010
:10220000286A40F004002862286A40F00100C1E713
:10221000FFF7C4FB4FEA000897FAA7F0B0FA80F086
:1022200040F04000B6EB501F08BF28680AD097FA6C
:10223000A7F0B0FA80F040F04000B7EB501F0CBFA1
:10224000286A686A97FAA7F1B1FA81F101F01F01D3
:1022500006FA01F1084206D0FFF7A0FBA0EB080048
:102260005045D9D93BE0BBF1000F03D0E86920F01D
:102270008050E861E069A8B3696801F00C010829A1
:102280007FD04FF0807A02289AFAAAF0B0FA80F054
:102290004FEA800000F1844000F584004FF00077A1
:1022A000C0F800901FD0FFF779FB044697FAA7F01B
:1022B000B0FA80F040F02000400914BF2868686A36
:1022C00097FAA7F1B1FA81F101F01F0106FA01F1C5
:1022D000084259D0FFF762FB001B0228E6D9032011
:1022E000BDE8F88F50E0FFF759FB804697FAA7F05A
:1022F000B0FA80F040F02000400914BF2868686AF6
:1023000097FAA7F1B1FA81F101F01F0106FA01F184
:10231000084206D0FFF742FBA0EB08000228E5D9EF
:10232000DDE7D4E908100843696821F47411084313
:1023300068609AFAAAF0B0FA80F0800000F1844058
:1023400000F584000660FFF729FB044697FAA7F022
:10235000B0FA80F040F02000400914BF2868686A95
:1023600097FAA7F1B1FA81F101F01F0106FA01F124
:10237000084209D1FFF712FB001B0228E6D9AEE79D
:10238000FFE70120BDE8F88F0020BDE8F88F4FF08F
:10239000E021042808690CBF40F0040020F004008C
:1023A0000861704770470000411EB1F1807F24BF73
:1023B000012070474FF0E0204161054AF02182F88A
:1023C000141D002181610721016100207047000078
:1023D0000FE000E010B5FFF7E5FF10BD7047704754
:1023E00090F83820012A04BF0220704710B401225F
:1023F00080F8382002685368D2F808C0A2F18044FF
:10240000B4F5963403D14C6823F4700323430C686D
:1024100023F07003896823432CF0800C41EA0C01FF
:10242000536002689160002180F8381010BC0846A3
:102430007047002804BF0120704710B5044690F88B
:10244000390028B9002084F83800204600F00CF844
:10245000022084F83900211D206800F011FB0120C2
:1024600084F83900002010BD38B5054600682549BC
:10247000B0F1804F25D0A0F18042B2F580520ED04D
:10248000A0F18042B2F5A05218BF38BDC86940F033
:102490002000C861C86900F02000009038BDC869FC
:1024A00040F01000C861C869002200F010000090E0
:1024B00011463620FFF7F6FABDE838403620FFF720
:1024C000E5BAC86940F00100C861C8690F4C00F066
:1024D000010000900C4820601020606000208021E6
:1024E000C4E9020120616061A0614FF44050E061E5
:1024F0002046FEF7BFFF002818BFFEF750FA2C62F7
:10250000656238BD001002405800024020020020E1
:10251000022180F8391001680A6842F001020A605D
:10252000012180F839100020704790F83820012AE6
:102530000DBF0220012380F83830704730B40222EA
:1025400080F839200268D2F808C02CF0770C2CF4FF
:10255000803C2CF47F4CC2F808C00A68502A47D04F
:102560000CDC202A7DD004DC002A7BD0102A7AD013
:10257000B7E0302A78D0402A78D0B2E0602A54D030
:10258000702A0DD0B2F5805F03D0B2F5005F1DD088
:10259000A7E001688A6822F0070222F4803242E054
:1025A0000268D1F804C08C68C96895684CEA0121BA
:1025B00025F47F4521432943916001688A6822F010
:1025C000770222F4803242F077022CE00268D1F8E0
:1025D00004C08C68C96895684CEA012125F47F45E0
:1025E00021432943916001688A6842F480421AE0DD
:1025F0000268D1F804C0C968146A156A25F001059B
:102600001562956924F00A0425F0F00545EA0111E8
:1026100044EA0C0C9161C2F820C001688A6822F07B
:10262000700242F057028A605BE00268D1F804C091
:10263000CC68116A21F0100111629569116A25F4C4
:10264000704545EA043421F0A00141EA0C1194617F
:10265000116201688A6822F0700242F067028A60A3
:102660003FE02FE01EE025E034E0FFE70268D1F80C
:1026700004C0CC68116A156A25F0010515629569D8
:1026800021F00A0125F0F00545EA041441EA0C01A5
:102690009461116201688A6822F0700242F0470278
:1026A0008A601EE001688A6822F0700242F0070228
:1026B0008A6016E001688A6822F0700242F0170210
:1026C0008A600EE001688A6822F0700242F02702F8
:1026D0008A6006E001688A6822F0700242F03702E0
:1026E0008A6080F83930002180F8381030BC084604
:1026F0007047704770B50446006801694FF00005E7
:1027000011F0020F1CBFC16811F0020F13D06FF05F
:1027100002010161012020762068806910F0030F1A
:10272000204602D0FFF7E5FF04E000F035F920462F
:1027300000F04FF925762068016911F0040F1CBFE5
:10274000C16811F0040F13D06FF004010161022081
:1027500020762068806910F4407F204602D0FFF781
:10276000C8FF04E000F018F9204600F032F92576A1
:102770002068016911F0080F1CBFC16811F0080F33
:1027800013D06FF008010161042020762068C06931
:1027900010F0030F204602D0FFF7ABFF04E000F07B
:1027A000FBF8204600F015F925762068016911F044
:1027B000100F1CBFC16811F0100F13D06FF0100183
:1027C0000161082020762068C06910F4407F20460F
:1027D00002D0FFF78EFF04E000F0DEF8204600F0A4
:1027E000F8F825762068016911F0010F1CBFC16857
:1027F00011F0010F05D06FF001010161204600F0DA
:10280000E9F82068016911F0800F1CBFC16811F060
:10281000800F05D06FF0800101612046FFF7DEFDDB
:102820002068016911F0400F1CBFC16811F0400F12
:1028300005D06FF040010161204600F0D9F8206812
:10284000016911F0200F1ABFC16811F0200F70BD8F
:102850006FF0200101612046BDE87040FFF7BFBD69
:102860002DE9F047044690F8380001280DBF0220FA
:10287000012584F83850BDE8F087022084F839003B
:102880000C2A1BD008DC8AB1042A13D0082A04BF02
:10289000206800F0D1F96EE03B4BDFF8F0C03C4E11
:1028A0003C4F102A0ED0142A39D064E0206800F082
:1028B00039F960E0206800F07FF95CE0206800F002
:1028C000FBF958E02268106A20F480301062D2F8D8
:1028D00020905068D2F85480D1F800A028F07008F9
:1028E00028F480384AEA0808B1F808A029F4003929
:1028F00049EA0A499A4218BF624503D0B24218BF5A
:10290000BA4204D14B6920F4803040EA0320506081
:10291000C2F8548048689065C2F820902BE0226885
:10292000106A20F480101062D2F820805068D2F82B
:102930005490D1F800A029F4E04929F0807949EABF
:102940000A29B1F808A028F4001848EA0A589A425F
:1029500018BF624503D0B24218BFBA4204D14B69D6
:1029600020F4802040EA83205060C2F854904868E8
:10297000D065C2F8208084F839504FF0000084F808
:102980003800BDE8F0870000002C01400040014005
:1029900000440140004801407047002804BF012066
:1029A000704710B5044690F8390028B9002084F823
:1029B0003800204600F00CF8022084F83900211D70
:1029C000206800F05DF8012084F83900002010BD77
:1029D000704770470449884218BF70470348016830
:1029E000491C016070470000A8010020C4000020BD
:1029F0007047FF2000F08AFDFEE7FEE7704710B544
:102A0000FEF7D2FFBDE81040FFF7E4BC14480168B0
:102A100041F4700101601348016841F00101016057
:102A20004168114A11404160016821F4102121F0F0
:102A300080710160016821F480210160416821F406
:102A4000FE014160C16A21F00F01C162016B074ABA
:102A500011400163002181600549C003086070478F
:102A600088ED00E0001002400CC07FF8CCFC00FFB5
:102A700008ED00E00148FFF73DBE0000A80100207E
:102A800070B402681B4B1C4E98421CBFB0F1804FC3
:102A9000B04205D1D1F804C022F070024CEA020223
:102AA000DFF858C0164C174D984218BFB0F1804F50
:102AB00007D0B04218BF604503D0A04218BFA8425B
:102AC00004D1CE6822F4407246EA020202608A68AB
:102AD000C2620A688262984218BF604503D0A04271
:102AE00018BFA84201D1096901634FF0010141619A
:102AF00070BC7047002C01400004004000400140C1
:102B000000440140004801400123D0F820C08B4020
:102B10002CEA03030362036A02FA01F1194301621A
:102B2000704700002DE9F001026A22F00102026202
:102B3000026A4368D0F818C00C682CF0730C2CF4AF
:102B4000803C44EA0C0C8C6822F002022243164CB2
:102B5000164D174E174FA04218BFA84203D0B042DF
:102B600018BFB84207D1D1F80C8022F0080248EA19
:102B7000020222F00402A04218BFA84203D0B042D1
:102B800018BFB84207D14C6923F4407344EA0303E9
:102B90008C6944EA03034360C0F818C04968416384
:102BA0000262BDE8F0017047002C01400040014086
:102BB000004401400048014010B4026A22F01002B3
:102BC0000262026A4368D0F818C00C682CF4E64C24
:102BD0002CF0807C4CEA042C8C6822F0200242EA23
:102BE0000412A0F18044B4F596340ED0A0F18044D4
:102BF000B4F5A0341FBFA0F18044B4F5A234A0F115
:102C00008044B4F5A43407D00EE0CC6822F08002F2
:102C100042EA041222F040024C6923F4406343EA82
:102C200084038C6943EA84034360C0F818C0496890
:102C30008163026210BC704710B4026A22F4807291
:102C40000262026A4368D0F81CC00C682CF0730C56
:102C50002CF4803C44EA0C0C8C6822F4007242EAAA
:102C60000422A0F18044B4F596340ED0A0F1804443
:102C7000B4F5A0341FBFA0F18044B4F5A234A0F194
:102C80008044B4F5A43407D00EE0CC6822F400628E
:102C900042EA042222F480624C6923F4405343EA5E
:102CA00004138C6943EA04134360C0F81CC04968EC
:102CB000C163026210BC704710B4026A22F48052F1
:102CC0000262D0F820C04268C3690C6823F4E6436E
:102CD00023F0807343EA04238C682CF4005C4CEAF4
:102CE000043CA0F18044B4F596341CBFA0F18044AC
:102CF000B4F5A03409D0A0F18044B4F5A2341CBFCF
:102D0000A0F18044B4F5A43404D14C6922F480428B
:102D100042EA84124260C36149680164C0F820C07D
:102D200010BC7047FEE703B401984100009850EAD8
:102D3000C12018BF04204A0D18BF40F0010040F226
:102D4000FF72B2EB515F08BF40F00200012808BFDC
:102D5000052002B07047000070B52DED020B2DED7F
:102D60000A8B82B00D98C40F20F00045AE48854212
:102D700048D3AE48854219D30C99C5F313000843D4
:102D800009D09DED0C0B02B0BDEC0A8B02B0BDE882
:102D9000704000F046BA002C14BF9FEDA50B9DEDCE
:102DA0000C0B02B0BDEC0A8B02B070BD9FEDA20B04
:102DB00053EC102B9DED0C0B51EC100BFDF746FD69
:102DC0000AD2022000F068FA02B0BDEC0A8B02B011
:102DD000BDE8704000F030BA9FED990B53EC102B1A
:102DE0009DED0C0B51EC100BFDF718FD0AD20220E3
:102DF00000F052FA02B0BDEC0A8B02B0BDE87040A0
:102E000000F02ABA90489FED92BBA8425CD292484B
:102E1000854219D29148784400EBC40090ED000B34
:102E200053EC102B9DED0C0B51EC100BFDF79DFAA4
:102E300041EC1A0B8A48784400EBC40090ED009BEB
:102E4000C4F10100041B36E09FED870B53EC102BFF
:102E50009DED0C0B51EC100BFDF78DFA41EC100BB6
:102E60008348784400EBC40090ED001B51EC100B3C
:102E700053EC112BFDF7D8F9FDF7B1FC0446FDF733
:102E80009DFC41EC180B9FED7C0B53EC102BFDF7D8
:102E900072FA9DED0C1B53EC112BFDF769FA41EC16
:102EA0001A0B9FED770B51EC180B53EC102BFDF721
:102EB00062FA41EC190B51EC1A0B53EC192BFDF78C
:102EC00054FACDE90C011BE06F48854217D29FED03
:102ED000700B53EC102B9DED0C0B51EC100BFDF710
:102EE000A3F953EC1B2BFDF7B1FC08D29DED0C0BA5
:102EF00053EC1B2B51EC100BFDF796F96EE0002400
:102F00009DED0C0B53EC102B51EC100BFDF733FA2D
:102F100041EC180B60480521B0EE480AF0EE680A53
:102F2000784400F002F953EC182B51EC100BFDF72C
:102F300022FA9DED0C1B53EC112BFDF719FA41EC15
:102F4000180B9FED570B5CB353EC182B51EC100B87
:102F5000FDF70BFA9DED0C0B41EC1C0B53EC182B01
:102F600051EC100BFDF707FA53EC1C2BFDF775FA2B
:102F700053EC192BFDF7FCF953EC1A2BFDF7F5F97F
:102F800053EC1B2BFDF7F4F9CDE900016FF47F70D2
:102F9000844226DB01EB045001909DED000B00E71D
:102FA00053EC102B51EC180BFDF7DFF99DED0C0BDA
:102FB00041EC190B53EC182B51EC100BFDF7DBF91E
:102FC00053EC192BFDF749FA9DED0C1B53EC112B1B
:102FD000FDF7CBF953EC1B2BFDF7CAF941EC100BB5
:102FE000DFE608464FF07A5101EB04519FED2E0BBE
:102FF000084453EC102B01909DED000B51EC100B8D
:10300000FDF7B9F90D4645EC100B044651EC100BD9
:10301000FFF789FE042808BF00F01EF945EC104BAD
:10302000BFE6000000000000422E86400000F07F56
:103030000000000000000000EF39FAFE422E86403A
:1030400051302DD5104987C0422ED63F00000000D8
:10305000000000000000F03FB2A2F03F8614000024
:103060007614000000000000FE822B654715F73F34
:103070002A140000000000000000E0FE422EE63F9F
:10308000763C7935EF39EA3D0000303E0000000023
:103090009C7500883CE4377E9C1300000000000013
:1030A000000000000000004000000000000070016F
:1030B00000B52DED048BB0EE409AF0EE609A83B02F
:1030C00051EC190BFDF729FB41EC180B18EE100A17
:1030D00018EE901A8DED008B002818BF01200843D0
:1030E00020F00040C0F17F6000F1E040C00F14D03C
:1030F00019EE101A19EE900A8DED009B002918BFE9
:103100000121084320F00040C0F17F6000F1E04061
:10311000C00F04BF012000F0BFF8B0EE480A03B0B2
:10312000F0EE680ABDEC048B00BD70B504462DEDD1
:10313000028B4D1E00EBC500B0EE408AF0EE608AB7
:1031400090ED000B35F0060017D053EC182B51EC26
:10315000100BFDF710F941EC100B6D1E04EBC500D0
:1031600090ED001B51EC100B53EC112BFDF75CF8AC
:1031700041EC100B35F00600E7D1022D36D0042DBE
:103180001CD0062D1CBFBDEC028B70BD53EC182B60
:1031900051EC100BFDF7EFF894ED0A1B53EC112BDB
:1031A000FDF742F853EC182BFDF7E5F894ED081BFA
:1031B00053EC112BFDF738F841EC100B53EC182BA6
:1031C00051EC100BFDF7D7F894ED061B53EC112BC7
:1031D000FDF72AF853EC182BFDF7CDF894ED040B0E
:1031E00053EC102BFDF720F841EC100B53EC182B8F
:1031F00051EC100BFDF7BFF894ED021B53EC112BB3
:10320000FDF712F853EC182BFDF7B5F894ED001B01
:1032100053EC112BFDF708F8BDEC028B41EC100BC1
:1032200070BD10B553EC102B51EC100BFCF7FCFFEC
:1032300041EC100B10BD00009FED050B10B553ECD9
:10324000102B51EC100BFDF796F841EC100B10BD54
:1032500000000000000000709FED050B10B553EC5E
:10326000102B51EC100BFDF786F841EC100B10BD44
:10327000000000000000001002E008C8121F08C192
:10328000002AFAD170477047002001E001C1121FE7
:10329000002AFBD170470000014908607047000018
:1032A000140100202DE9F0410026144F144C35463E
:1032B000012208213846FEF76CFBFA235FF000027A
:1032C0004FF47A71256020688842FCD3521C9A42E0
:1032D000F6DB002208213846FEF75BFBFA230021CB
:1032E0004FF47A72256020689042FCD3491C9942C1
:1032F000F6DB761C022EDBDBBDE8F0810004004823
:10330000241400402DE9F0470E462DED028B0546B2
:10331000B0EE408A10216E48FEF732FB012818BF3C
:1033200000206C4C94ED040ADFED6B0A60EE200A7D
:1033300000EE100AB8EE400A9FED681A684A40EEA7
:10334000010AC4ED040A94ED050A30EEC00AB0EE9D
:10335000C00A10EE101A91422CDD10EE901AB1F155
:103360007C5FD4BF9FED5F0AB7EE000A84ED040ACC
:10337000B5EEC00A84ED050AF1EE10FA1AD15A4FE3
:103380003868152808BFFEF7D1FB584B38681A4635
:103390000021401CE0FB03210909A1EBC10101EB65
:1033A0004101081808BF012030600220286084ED28
:1033B000068A71E0002818BF84ED068A4FD04C4879
:1033C000FDF7DEFF05214A48FDF75AFFDFF820919F
:1033D000002856D0112000F099F805214448FDF747
:1033E0004FFF002853D0122000F090F800EE908A92
:1033F00094ED000A9FED3F1AF8EE600ADFED3E1AE9
:1034000020EE010A9FED3D2A60EEA10A3C4800EE45
:10341000820A84ED000AD4ED020A60EE810A01EE10
:10342000107AB8EE411A21EE211A41EE020AC4EDDB
:10343000020A94ED011A30EE411AB0EEC11A11EEF3
:10344000101A81422DDD84ED010ADFED2E0A0320E2
:1034500020EE200ABCEEC00A86ED000A35E094EDAD
:10346000060A38EE400A10EE100AB0F1804FA6DDD1
:1034700005209FED250A286038EE000A84ED060A33
:103480000AE0D9F80000006C1FFA80F8A5E7D9F827
:103490000000006C87B2A9E7BDEC028B0120BDE8FB
:1034A000F08794ED030A30EEC00AB0EEC00A10EEC9
:1034B000101A8142DEBF0020BDEC028BBDE8F08710
:1034C000C4ED030AC6ED000A01202860E4E700000D
:1034D00000040048F80000203333333F9A99993EA6
:1034E000CDCC4C3F0000000034000020C3300CC3A2
:1034F000180100206666663FD0CCCC3D00008039C4
:103500000AD7233C00007F430000C8422DE9F04762
:103510000027DFF8FC903F4C80464FF0010A3D4603
:10352000012208214846FEF734FA28225FF0000104
:103530004FF47A70256023688342FCD3491C914282
:10354000F6DB002208214846FEF723FA1422002069
:103550004FF47A71256023688B42FCD3401C904263
:10356000F6DB012208214846FEF713FA2822002044
:103570004FF47A71256023688B42FCD3401C904243
:10358000F6DB002208214846FEF703FA4FF4C87222
:103590005FF000004FF47A71256023688B42FCD302
:1035A000401C9042F6DB0026C6F107000AFA00F044
:1035B00010EA080F04D0012208214846FEF7E9F975
:1035C000642300214FF47A70256022688242FCD384
:1035D000491C9942F6DB002208214846FEF7D9F93A
:1035E0004FF4C8725FF000004FF47A7125602368D1
:1035F0008B42FCD3401C9042F6DB761C082ED3DBBA
:103600007F1C142F8CDBBDE8F047FEF78FBA00005B
:10361000000400482414004010B54FF090430022ED
:103620005A61014640F6C9330A4A0B48FEF776F85C
:103630000A4C2068C16841F40071C1600122002178
:103640009007FFF761FA2068016841F0010101600D
:1036500010BD000014000048200200206C01002072
:1036600010B5002211464FF08040FFF74DFA134984
:103670000868036A41F21112134240F2444304BF46
:10368000D0F820C01CEA030F05D1D0F844C02CF4B8
:10369000004CC0F844C0D0F820C01CEA020F04BFA0
:1036A000026A1A4203D1026822F00102026008682D
:1036B000C16821F40071C16010BD00006C010020E0
:1036C00010B5142200211A48FDF704FF20B1BDE80F
:1036D00010400820FFF71ABF002211464FF080402B
:1036E000FFF712FA13490868036A41F211121342F4
:1036F00040F2444304BFD0F820C01CEA030F05D1B8
:10370000D0F844C02CF4004CC0F844C0D0F820C01D
:103710001CEA020F04BF026A1A4203D1026822F0B7
:10372000010202600868C16821F40071C16010BD27
:10373000200200206C01002091F800C04A788B78AC
:103740005FF0280100F801CB491E00F8012B00F8BA
:10375000013BF7D1002070470C48016821F00101BE
:103760000160416A0A4A89B292ED000A026842F099
:103770000102026000EE901AB8EE400A9FED051AB1
:10378000F8EE600A00EE810A704700000010004069
:10379000C400002017B7D1382DE9F04116460F4676
:1037A00016287DD2DFE800F0950B0B0B0B0B0B11ED
:1037B0001D222F0B0B0B0B0B0B0B0B0B0B3FC1B27B
:1037C0003846FDF76DF8014632E0B0083D46282145
:1037D00005F8016B491E05F8010B05F8016BF7D1DF
:1037E00026E038467821FCF70DFD1AE0B0083C468B
:1037F0005FF0280104F8016B491E04F8016B04F81E
:10380000010BF7D114E078213846FCF702FD3E7039
:10381000FE7087F8286087F82B6087F8536087F878
:103820005660002104E038467821FCF7F2FC0021C4
:103830000020FB1E844602461424DD7893F80480A1
:10384000641E454493F80580C444AC4413F8065FF5
:103850001FFA8CFC93F80180454493F8028042449F
:103860002A4492B2E9D1624492B2824288BF1046A1
:10387000C6EB0612D200904228DD00EE102ADFEDE2
:10388000160AB8EEC00A60EE200A00EE100AB8EE82
:10389000400A80EE801ABCEEC10A10EE100A00E069
:1038A00017E082B2781E3C2310F801CF5B1E0CFBA0
:1038B00002FC4FEA1C2C00F801CB90F800C00CFB76
:1038C00002FC4FEA1C2C80F800C0EDD10846BDE890
:1038D000F0810020BDE8F0810000804301464FF4F4
:1038E000707200234FF0FF0C01F801CB521E01F85B
:1038F000013B01F8013BF7D1892100F53460FCF769
:1039000088BC0000000000002DED0A8B90B04FF045
:10391000904B0025FD4CFC48206000F6C9306060EB
:10392000CBF81450FEF748F84FF46010CDE908507A
:1039300002264FF001084FF01009009607966846DE
:10394000CDE90489FEF742FA00B1FEE70F20CDE988
:103950000B064FF48060CDE90D5002210BA80F95A6
:10396000FEF706F900B1FEE7FEF72AFA4FF47A7186
:10397000B0FBF1F0FEF718FD0420FEF708FD002271
:103980001146501EFEF78EF8E14F786940F4003082
:103990007861786900F400300590786940F48020FF
:1039A00078617869002200F48020059001214FF0B1
:1039B0009040FDF7EEFFDFF85CA30022082150469F
:1039C000FDF7E7FFCDF80080CDE9018569464FF0AE
:1039D00090400395FDF7D2FE08200090CDE90185C7
:1039E000694650460395FDF7C9FECDF80090CDE934
:1039F000015869465046FDF7C1FE786940F0010064
:103A000078617869002200F00100009011460F20D3
:103A1000FEF748F80F20FEF739F8C048BE4F4FF4C4
:103A2000C8510760C0E9011542F20F71C160FEF78D
:103A300000FD00B1FEE700956946B8480295FEF723
:103A4000CFFC00B1FEE7B748B5494FF04009C0E9E7
:103A500000194FF6FF71C0E90251FEF7EAFC00B110
:103A6000FEE700956946AF480295FEF7B9FC00B144
:103A7000FEE7AD484FF08041C0E900151921C0E9CB
:103A800002510561FEF7D5FC00B1FEE74FF480500E
:103A90000C900CA9A448FEF748FD00B1FEE7A2482F
:103AA000FEF77BFF00B1FEE7079507A99E48099541
:103AB000FEF796FC00B1FEE7302000900A20CDE929
:103AC00001050022694698480495FEF7C9FE00B139
:103AD000FEE796484FF0A04101604FF44031C0E945
:103AE0000115C561456206620563C0E90358456377
:103AF00004218563C0E90518FDF77CFA00B1FEE7F3
:103B00000B20CDE900080320CDE9020504956946A4
:103B100086480595FCF748FF00B1FEE70C20CDE98B
:103B2000000669468148FCF73FFF00B1FEE7CBF88D
:103B300014507F4880687E4940F0010088608868A2
:103B400040F010017A488160806840F02001784898
:103B500081607248FEF7DCFC7248FEF7D9FCFFF783
:103B6000A1FB7448802101704021417081700146A1
:103B70007148FFF7E1FD3620FDF77CFF0222114678
:103B80003620FDF78FFF3D613620FDF77FFFF86897
:103B900040F00100F8604FF0010B4FF00009206881
:103BA000FFF79CFE6068FFF799FE644EF7EE009AFF
:103BB0003220C6F82C8086F80280F070B0EE698A58
:103BC000FFF7CAFD86ED0C0AF0EE408A9FED5C9A85
:103BD000F0EE490AB0EE490A00F048FAB0EE490AA0
:103BE00000F000FA574F9FED58CADFED58CA9FED1D
:103BF00058AB0024B0EE680A52490AA8FFF782FBCE
:103C000000281CBFB2EE02BADFED53BA61D00A98A9
:103C10000124062855D2DFE800F0030C174030439A
:103C200097ED000A00F0DEF908215046FDF7ADFEE1
:103C300047E097ED000AB0EE698A082100EE0B8A92
:103C40005046FDF7A2FE3CE03868B0EE490AF0624B
:103C500000F0C8F9F06AD6ED0C0A0A280CBFB0EEE5
:103C60006B0AB0EE490A00F001FA00BF86F8028044
:103C700008215046FDF789FE23E032497822A1F160
:103C8000F000FCF7ADFA80212B48F56200F060F9F6
:103C900008215046FDF779FE13E03878F070E5E72B
:103CA000FFF70EFD1848FFF719FE1748FFF7B4FCA1
:103CB000142200212948FDF70DFCFFF7D1FCFDF788
:103CC00047FFB0EE680A1F490AA8FFF71BFB002850
:103CD0009DD1B0EE68BAFFF73FFDF0EE408A96ED59
:103CE0000C0A78EECB0A00EE880A86ED0C0A00F08A
:103CF0000DFA86ED080A3078B0EE680A90BB1848D5
:103D0000002150F8043B2EE0C40300203C000020BA
:103D1000001002400004004800100040A8010020EC
:103D200000140040E40100206C0100201801002074
:103D3000002004E0100000205C02002008000020A9
:103D4000000000004C030020CDCCCC3C3333333F8B
:103D50000000000080842E41CDCCCC3D200200200C
:103D60004400002031E0C3EB031301EB830140F872
:103D7000041C50F8083B0E22C3EB031301EB830134
:103D800040F8081C50F8043CC3EB031301EB83011B
:103D900040F8041C0368C3EB031301EB83010160CB
:103DA00050F8043F521EC3EB031301EB830140F8AC
:103DB000041B0368C3EB031301EB83010160EFD124
:103DC000501E7161F06086F80080002C1CBF86EDEB
:103DD000040A757042D1D6ED040A30EE600ABCEEDA
:103DE000C00A10EE100AB0F5616F8CBF01210021EE
:103DF0007278114332D07169B0FBF1F201FB12010C
:103E00004020F0704C4A002052F820308B420AD8F3
:103E100002EB80035B688B4201D9401C03E0801CED
:103E20002028F1DB0A204549085CF062D6ED0C0A37
:103E30000A2857D0B0EE490A00F018F9B0EE490A46
:103E400000F0D0F8F16AF068814205D014281CBF58
:103E50001420F06286F80280F06AF060D6ED080A5D
:103E6000BDEEE00A10EE100AB06200EE100AB8EEE5
:103E7000C00A30EEC00A10EE101A86ED090AB1F140
:103E80007C5F08DD30EE690A401C282886ED090AAF
:103E9000B06208BFB562F06A00281CBFB178002983
:103EA00006D0F27896ED0C0A2549FFF775FCB07044
:103EB00096ED090A234B0121F1EE400AA3F17802A5
:103EC0002820B0EE6C0AFCF7F0FC1F4850F82910CF
:103ED000F16196F828201B48FCF7ECFCBBF1000FC1
:103EE0000AD104E0B0EE4C0A00F0C0F8AAE7FFF7F0
:103EF000E7FB16480068F080F069FFF78DFB134878
:103F000042F21072016889B2B1809142FAD3056021
:103F1000B088FCF711FB41EC100B51EC1A0B53EC81
:103F2000102BFCF79AFAFCF727FB4FF0000BC9F1B6
:103F30000109B0615DE6000044000020B4410008C2
:103F40005C020020D40200203C0000202414004029
:103F5000F0B44FF0000CC21E654664461423D678B8
:103F600017795B1E3E4457793D44354412F8066F7D
:103F7000ADB257783E4497783C443444A4B2EED175
:103F80002A1992B2624588BF9446C1EB0111C9005B
:103F90008C45DCBFF0BC704700EE101A3C22B0F13B
:103FA0000100B8EEC00ADFED0E0A60EE200A00EE56
:103FB00010CAB8EE400A80EE801ABCEEC10A10EEBC
:103FC000101A89B210F8013F4B431B0A00F8013B5D
:103FD00003784B431B0A0370521EF3D1F0BC7047A9
:103FE0000000804310EE100ADFED1B0A10F1814F34
:103FF00004D210EE100AB0F17E5F02DBB0EE600A70
:1040000008E0B5EEC00AF1EE10FA3CBFF7EE000A88
:1040100030EE200ADFED110A1149124820EE200A85
:1040200081ED020A026822F001020260426A91ED0B
:10403000000A036892B243F001030360F8EE400AFD
:1040400000EE102A9FED081AB8EE400A40EE010A71
:10405000C1ED030A7047000000000000000020428C
:10406000C40000200010004017B7D138244ADFED0B
:10407000251A92ED012AB5EEC02AF1EE10FA26D0EB
:1040800092ED031A204870EEC12A92ED021A02EE58
:10409000821A11EE101A82ED021A884208DC00BF63
:1040A00031EE611A11EE101A8142F9DA82ED021A2C
:1040B000B5EEC01AF1EE10FA09D200BF31EE211AA6
:1040C000B5EEC01AF1EE10FAF8D382ED021A10EE36
:1040D000100AC2ED030AB0F17E5F0ADC10EE100A8E
:1040E00010F1814F08D800BF20EE210A82ED010AAD
:1040F0007047B7EE000AF7E7BFEE000AF4E70000EA
:10410000C400002000002042000020421A4AB0EE05
:10411000401A1046D2ED010A90ED020AF5EEC00AEF
:10412000F1EE10FA25D0D2ED031A144871EE611A9F
:1041300001EEA00ADFED120A10EE101A82ED020A5B
:10414000884207DC30EE600A10EE101A8142F9DA7C
:1041500082ED020AB5EEC00AF1EE10FA09D200BFF4
:1041600030EE200AB5EEC00AF1EE10FAF8D382ED77
:10417000020A82ED031A7047C400002000002042AA
:104180000000204202030405060708090A0B0C0D73
:104190000E0F10100102030405060708090A0B0C94
:1041A0000D0E0F10000000000000000001020304CB
:1041B000060708090A010A130A020A140A030A0573
:1041C0000A040A0C0A010A0D0A020A0E0A100A0F52
:1041D0000A110A12FF02020000003B027704B20635
:1041E000ED08270B610D990FD011051439166C18C5
:1041F0009C1ACA1CF71E202147236C258D27AB294A
:10420000C62BDE2DF22F03320F3417361C381B3A23
:10421000173C0D3EFF3FEC41D343B64593476A49F7
:104220003B4B074DCD4E8C504652F953A5554B573D
:10423000E958815A125C9C5D1E5F99600C6278633C
:10424000DC6438668D67D9681D6A586B8B6CB66DF7
:10425000D96EF26F03710B720A730074EE74D2752B
:10426000AD767E7746780579BB79677A097BA27B44
:10427000317CB77C327DA47D0D7E6B7EC07E0A7F53
:104280004B7F827FAF7FD27FEB7FFA7FFF7F000083
:10429000000000000000E03F000000000000E0BF60
:1042A0000000E0FE422EE63F0000E0FE422EE6BFA8
:1042B000763C7935EF39EA3D763C7935EF39EABD20
:1042C0003E5555555555C53F93BDBE166CC166BF8D
:1042D0002CDE25AF6A56113FF16BD2C541BDBBBE86
:1042E000D0A4BE726937663E184300080000002063
:1042F0001801000078320008304400080000001067
:10430000D808000078320008304400081801002066
:10431000A01C0000883200080000000000127A0093
:10432000000100000000000000000000000000008C
:10433000000000000000000000000000000000007D
:10434000000000000000000000000000000000006D
:10435000000000000000000000000000010000005C
:104360000A000000020000000A0000000200000035
:104370000A000000010000000A0000000100000027
:104380000A000000020000000A0000000200000015
:104390000A000000010000000A0000000100000007
:1043A0000A000000020000000A00000002000000F5
:1043B0000A000000010000000A00000001000000E7
:1043C0000A000000020000000A00000002000000D5
:1043D0000A000000010000000A00000000000000C8
:1043E00000000000000000000000000001000001CB
:1043F0000203040506070001020304050607000185
:104400000203040506070001020304050607000075
:1044100000000000000080BF00000000000080BF1E
:104420000000803F0000803F00000000000000000E
:1044300040F2535CC0F6000C604742F6595CC0F68F
:10444000000C604743F2B10CC0F6000C604740F22C
:10445000773CC0F6000C604740F25B4CC0F6000CA5
:10446000604740F2795CC0F6000C604740F2292CAE
:10447000C0F6000C6047000010B560EEE00A2DEDBC
:10448000048BB0EE408AB0EE000A28EE000A20EE5F
:10449000081A80EE810A10EE100AFFF7C9FF41ECFE
:1044A000100BFFF7CAFFB0EE409AF0EE609A18EEDC
:1044B000100AFFF7BDFF41EC180B9FED830BFFF7D0
:1044C000C1FF53EC182B51EC100BFFF7C0FF41EC70
:1044D000100B53EC102B9FED7E0B51EC100BFFF7E4
:1044E000BBFF53EC192BFFF7B2FFFFF7BAFFBDEC90
:1044F000048B00EE100A10BD2DE9F04107462DEDAA
:10450000108B481E00EBD070B0EE41EAF0EE608AEE
:10451000B0EE40FA4610DFED709A75423C46B0EEC0
:10452000698AB54250DCB0EE000A28EE800A60EEDF
:1045300028EA9FED65DB9FED66CBDFF8A08100BF29
:1045400000EE105AB0EE4E9AB8EEC00A00EE0F9A86
:1045500069EE490A80EEAE0A10EE100AFFF768FF16
:1045600041EC100BFFF769FFB0EE40AAF0EE60AA35
:1045700018EE900AFFF75CFF41EC1B0BB0EE4D0A02
:10458000F0EE6D0AFFF75EFF53EC1B2B51EC100BA6
:10459000FFF75DFF41EC100B51EC1C0B53EC102BA3
:1045A000FFF75AFF53EC1A2BFFF751FFFFF759FFA4
:1045B00020604045B8BFC4ED009AB4EC010A6D1C00
:1045C000B54230EE088ABBDD012000EB4601002930
:1045D000DCBFBDEC108BBDE8F081384697ED000ADA
:1045E0004910C0EE080AC7ED000A0ED090ED010A8E
:1045F000C0EE080AC0ED010A90ED020AC0EE080AFA
:10460000C0ED020A0830491EF0D1BDEC108BBDE8A8
:10461000F081F0B5B0EE601A85B0F0EE400A1E46AB
:104620001446B7EE000A05216846FFF765FF002330
:10463000DFED292A194600BFB0EE621A0022F0EE23
:10464000410AB0EE410AEC4605258818801E48BF95
:10465000283002D42828A8BF283800EB4000DCED21
:10466000001A275C401C02EE107A275C2044B8EE4A
:10467000422A4078521C6D1E01EE820A02EE107A28
:104680000CF1040CB8EE422A41EE820A02EE100A46
:10469000B8EE422A01EE821AD7D1BCEEC00A491CFC
:1046A00010EE100ABCEEE00AF054F01810EE102ADA
:1046B000BCEEC10A4270DB1C10EE102A2829827061
:1046C000BADB05B0F0BD000000000060FB2119401E
:1046D000000000000000F03F000000000AD7233C6B
:1046E0002DE9F04F07462DED0E8B0D4683B0904619
:1046F000F748017800291CBF00210170F2EE040A7E
:10470000F1EE00AA80EE209A00209FEDF20AF6EE6C
:10471000008A064630EE680A00EB800B2AEE80AA7B
:104720009FEDED0A69EE00CA29EE28CADFEDEBDA4B
:10473000B7EE00EA00EE106AF0EE6ABA06EBCB00C4
:10474000F8EE400A00EB4004B0EE6ABAF0EE4A9A86
:1047500080EEAD0A30EE680A2BEE808A38EE090A48
:1047600000F03AFAB0EE40DA39EE890A20EE280A73
:1047700000F032FA30EE0DDA38EE290A30EE090A8E
:1047800020EE280A00F028FA30EE0DDAB0EE6C0ABE
:1047900000F022FA6BEEA80A00EE808AB0EE4C0A16
:1047A00000F057FA6BEE280A19EE100A40EE809AD4
:1047B000FFF73EFE28EE080A41EC1B0B09EEA90AA2
:1047C00030EE0E0A10EE100AFFF732FE41EC100B2D
:1047D000FFF738FE53EC1B2B51EC100BFFF746FE96
:1047E000FFF73FFE00EE100A00F0F6F930EE0D0A7A
:1047F000152D60EE289A6ED2DFE805F06D0B3E3E77
:104800000B6D0B6D6D6D6D0B3E613E613E3E3E0B63
:104810000B00DFEDB3BA29EEAB0A00F0DDF99FED36
:10482000B1BAF0EE4B0A40EE0B0ABCEEE00A10EE15
:10483000100A00F0FF099FEDAC0A09EEAB0A00F088
:10484000CBF9F0EE4B0A40EE0B0ABCEEE00A10EE9C
:10485000100AC0B29FEDA50A019009EEAB0A00F064
:10486000BBF9F0EE4B0A40EE0B0ABCEEE00A10EE8C
:10487000100AC0B200902EE09FED990A29EE800A3E
:10488000B0EE40BA00F0A8F9DFED96BAF0EE6B0A90
:1048900040EE2B0ABCEEE00A10EE100AB0EE4B0A16
:1048A00000F0FF0900F0D5F9F0EE6B0A40EE2B0A9C
:1048B000BCEEE00A10EE100A00F0FF0A0BE0DFED9C
:1048C000880A9FED8A0A09EEA00A00F085F9B0EE89
:1048D000688A00EE288A152D80F0E880DFE805F070
:1048E000E60B4B723FA40BE6E6E6E60B7FBE99D2E1
:1048F000588C651D2E0019FB08F0000A38550199E7
:10490000601C11FB08F1090A3954009911FB08F1E8
:10491000090AA01C395400F0D0B8019810FB08F027
:10492000000A3855601C19FB08F1090A395400992E
:1049300011FB08F1090AA01C3954BEE0009810FBD5
:1049400008F0000A38550199601C11FB08F1090AAA
:10495000395419FB08F1090AA01C3954ADE0601C58
:1049600007F8048007F80080009911FB08F1090A94
:10497000A01C3954A1E019FB08F0000A3855601C4E
:104980001AFB08F1090A39540021A01C395494E09B
:1049900000203855601C1AFB08F1090A395419FB2C
:1049A00008F1090AA01C395487E019FB08F0000A35
:1049B0003855601C002139541AFB08F1090AA01C63
:1049C00039547AE007F80480601C1AFB08F1090AE0
:1049D000395419FB08F1090AA01C39546DE019FB80
:1049E00008F0000A3855601C07F800801AFB08F12F
:1049F000090AA01C395460E019FB08F0000A385578
:104A0000601C1AFB08F1090A3954A01C07F8008041
:104A100053E007F80480601C19FB08F1090A3954B7
:104A2000A01C07F8008048E09FED310A29EE800ABB
:104A300000F0D2F8DFED2B0AB0EE601A00EE201A7B
:104A4000BCEEC10A10EE100AC0B210FB08F0000A5A
:104A5000611C38557854A11C78542EE000EE108A61
:104A600068EE080AB8EE400A20EE800ABCEEC00AE2
:104A700010EE100A3855601C07F80080A01C07F8DB
:104A800000801AE000EE108A68EE080A601CB8EE9A
:104A9000400A07F8048020EE800ABCEEC00A10EE3F
:104AA000101A3954A01C07F8008006E04FEA58019C
:104AB000601C39553954A01C3954761C282EFFF43B
:104AC00039AE03B00120BDEC0E8BBDE8F08F0000C5
:104AD000D4000020000000003BAAAA3E00002042B3
:104AE000DB0F49400000FF42920A0640920A8640CE
:104AF000DB0F49412DE9F84FDFF8CCA0DFF8CCC03F
:104B00009AF8003013BB0AF10109012799F8004017
:104B10004B4607FA04F5ACF8005099F8016064467A
:104B20005FF00F0513F8028F07FA06F6668007FAA2
:104B300008F85E7824F8048F6D1EF3D199F81F30C1
:104B400007FA03F3ACF83E308AF8007002EB420338
:104B500018444B1C4FF0000B1D4EDFF878E05D460B
:104B60006F46401C0BEB0201282908BF783800244F
:104B70005FF080018DF800508DF8015090F80080B2
:104B800018EA010F09D096F800809CF800A017F8E9
:104B9000089049EA0A0907F808909DF8008003F890
:104BA000038B4908E6D11EF904100844611CCCB2FD
:104BB000032CDDD30BF1010101F0FF0BBBF1280F3A
:104BC000D0D3BDE8F88F0000D5000020761B002070
:104BD000561B0020D4410008DFED460A20EE200AD3
:104BE000DFED450A4FF4B47180EE201ABDEEC10A24
:104BF00010EE100A90FBF1F201FB12000028B8BF82
:104C000000F5B4709FED3D0A3D49B0F5877FA8BF20
:104C1000C0F5B47014DAB4280CDB01EB4000A0F549
:104C20008050B0F8980E00EE900AF8EE600A20EE80
:104C3000800A70479FED330A5A28A8BFC0F1B4001C
:104C400031F8100000EE900AF8EE600A20EE800ABB
:104C50007047DFED280A4FF4B47120EE200ADFED33
:104C6000260A80EE201ABDEEC10A10EE100A90FB53
:104C7000F1F201FB12000028B8BF00F5B4709FEDFF
:104C8000210A1F49B0F5877F0CDB01EB4000A0F53E
:104C90008050B0F8E40D00EE900AF8EE600A20EEC5
:104CA000800A7047DFED150AB4280ADBC0F587706B
:104CB00031F8100000EE100AB8EE400A20EE200A8B
:104CC00070475A280ADB01EB400030F8B40C00EEC4
:104CD000100AB8EE400A20EE200A7047C0F15A00D0
:104CE00031F8100000EE900AF8EE600A20EE800A1B
:104CF0007047000000003443DB0F4940000100B85A
:084D0000D84100080001003851
:040000050800018965
:00000001FF
